C51 COMPILER V9.51   ADC_IRQ                                                               01/03/2014 20:23:49 PAGE 1   


C51 COMPILER V9.51, COMPILATION OF MODULE ADC_IRQ
OBJECT MODULE PLACED IN .\DP8051\DP8051_Keil_951\Debug\ADC_IRQ.obj
COMPILER INVOKED BY: C:\Program Files (x86)\Cypress\PSoC Creator\3.0\PSoC Creator\import\keil\pk51\9.51\C51\BIN\c51.exe 
                    -.\Generated_Source\PSoC3\ADC_IRQ.c NOIV LARGE MODDP2 OMF2 VB(1) PR(.\DP8051\DP8051_Keil_951\Debug\ADC_IRQ.lst) CD DB NOI
                    -P OT(2,SIZE) DF(DEBUG) INCDIR(.,.\Generated_Source\PSoC3) OJ(.\DP8051\DP8051_Keil_951\Debug\ADC_IRQ.obj)

line level    source

   1          /*******************************************************************************
   2          * File Name: ADC_IRQ.c  
   3          * Version 1.70
   4          *
   5          *  Description:
   6          *   API for controlling the state of an interrupt.
   7          *
   8          *
   9          *  Note:
  10          *
  11          ********************************************************************************
  12          * Copyright 2008-2012, Cypress Semiconductor Corporation.  All rights reserved.
  13          * You may use this file only in accordance with the license, terms, conditions, 
  14          * disclaimers, and limitations in the end user license agreement accompanying 
  15          * the software package with which this file was provided.
  16          *******************************************************************************/
  17          
  18          #include <cydevice_trm.h>
  19          #include <CyLib.h>
  20          #include <ADC_IRQ.h>
  21          
  22          #if !defined(ADC_IRQ__REMOVED) /* Check for removal by optimization */
  23          
  24          /*******************************************************************************
  25          *  Place your includes, defines and code here 
  26          ********************************************************************************/
  27          /* `#START ADC_IRQ_intc` */
  28          
  29          /* `#END` */
  30          
  31          
  32          /*******************************************************************************
  33          * Function Name: ADC_IRQ_Start
  34          ********************************************************************************
  35          *
  36          * Summary:
  37          *  Set up the interrupt and enable it.
  38          *
  39          * Parameters:  
  40          *   None
  41          *
  42          * Return:
  43          *   None
  44          *
  45          *******************************************************************************/
  46          void ADC_IRQ_Start(void) 
  47          {
  48   1          /* For all we know the interrupt is active. */
  49   1          ADC_IRQ_Disable();
  50   1      
  51   1          /* Set the ISR to point to the ADC_IRQ Interrupt. */
  52   1          ADC_IRQ_SetVector(&ADC_IRQ_Interrupt);
  53   1      
C51 COMPILER V9.51   ADC_IRQ                                                               01/03/2014 20:23:49 PAGE 2   

  54   1          /* Set the priority. */
  55   1          ADC_IRQ_SetPriority((uint8)ADC_IRQ_INTC_PRIOR_NUMBER);
  56   1      
  57   1          /* Enable it. */
  58   1          ADC_IRQ_Enable();
  59   1      }
  60          
  61          
  62          /*******************************************************************************
  63          * Function Name: ADC_IRQ_StartEx
  64          ********************************************************************************
  65          *
  66          * Summary:
  67          *  Set up the interrupt and enable it.
  68          *
  69          * Parameters:  
  70          *   address: Address of the ISR to set in the interrupt vector table.
  71          *
  72          * Return:
  73          *   None
  74          *
  75          *******************************************************************************/
  76          void ADC_IRQ_StartEx(cyisraddress address) 
  77          {
  78   1          /* For all we know the interrupt is active. */
  79   1          ADC_IRQ_Disable();
  80   1      
  81   1          /* Set the ISR to point to the ADC_IRQ Interrupt. */
  82   1          ADC_IRQ_SetVector(address);
  83   1      
  84   1          /* Set the priority. */
  85   1          ADC_IRQ_SetPriority((uint8)ADC_IRQ_INTC_PRIOR_NUMBER);
  86   1      
  87   1          /* Enable it. */
  88   1          ADC_IRQ_Enable();
  89   1      }
  90          
  91          
  92          /*******************************************************************************
  93          * Function Name: ADC_IRQ_Stop
  94          ********************************************************************************
  95          *
  96          * Summary:
  97          *   Disables and removes the interrupt.
  98          *
  99          * Parameters:  
 100          *   None
 101          *
 102          * Return:
 103          *   None
 104          *
 105          *******************************************************************************/
 106          void ADC_IRQ_Stop(void) 
 107          {
 108   1          /* Disable this interrupt. */
 109   1          ADC_IRQ_Disable();
 110   1      }
 111          
 112          
 113          /*******************************************************************************
 114          * Function Name: ADC_IRQ_Interrupt
 115          ********************************************************************************
C51 COMPILER V9.51   ADC_IRQ                                                               01/03/2014 20:23:49 PAGE 3   

 116          * Summary:
 117          *   The default Interrupt Service Routine for ADC_IRQ.
 118          *
 119          *   Add custom code between the coments to keep the next version of this file
 120          *   from over writting your code.
 121          *
 122          * Parameters:  
 123          *   None
 124          *
 125          * Return:
 126          *   None
 127          *
 128          *******************************************************************************/
 129          CY_ISR(ADC_IRQ_Interrupt)
 130          {
 131   1          /*  Place your Interrupt code here. */
 132   1          /* `#START ADC_IRQ_Interrupt` */
 133   1      
 134   1          /* `#END` */
 135   1      
 136   1          /* PSoC3 ES1, ES2 RTC ISR PATCH  */ 
 137   1          #if(CYDEV_CHIP_FAMILY_USED == CYDEV_CHIP_FAMILY_PSOC3)
 138   1              #if((CYDEV_CHIP_REVISION_USED <= CYDEV_CHIP_REVISION_3A_ES2) && (ADC_IRQ__ES2_PATCH ))      
                          ADC_IRQ_ISR_PATCH();
                      #endif /* CYDEV_CHIP_REVISION_USED */
 141   1          #endif /* (CYDEV_CHIP_FAMILY_USED == CYDEV_CHIP_FAMILY_PSOC3) */
 142   1      }
 143          
 144          
 145          /*******************************************************************************
 146          * Function Name: ADC_IRQ_SetVector
 147          ********************************************************************************
 148          *
 149          * Summary:
 150          *   Change the ISR vector for the Interrupt. Note calling ADC_IRQ_Start
 151          *   will override any effect this method would have had. To set the vector 
 152          *   before the component has been started use ADC_IRQ_StartEx instead.
 153          *
 154          * Parameters:
 155          *   address: Address of the ISR to set in the interrupt vector table.
 156          *
 157          * Return:
 158          *   None
 159          *
 160          *******************************************************************************/
 161          void ADC_IRQ_SetVector(cyisraddress address) 
 162          {
 163   1          CY_SET_REG16(ADC_IRQ_INTC_VECTOR, (uint16) address);
 164   1      }
 165          
 166          
 167          /*******************************************************************************
 168          * Function Name: ADC_IRQ_GetVector
 169          ********************************************************************************
 170          *
 171          * Summary:
 172          *   Gets the "address" of the current ISR vector for the Interrupt.
 173          *
 174          * Parameters:
 175          *   None
 176          *
 177          * Return:
C51 COMPILER V9.51   ADC_IRQ                                                               01/03/2014 20:23:49 PAGE 4   

 178          *   Address of the ISR in the interrupt vector table.
 179          *
 180          *******************************************************************************/
 181          cyisraddress ADC_IRQ_GetVector(void) 
 182          {
 183   1          return (cyisraddress) CY_GET_REG16(ADC_IRQ_INTC_VECTOR);
 184   1      }
 185          
 186          
 187          /*******************************************************************************
 188          * Function Name: ADC_IRQ_SetPriority
 189          ********************************************************************************
 190          *
 191          * Summary:
 192          *   Sets the Priority of the Interrupt. Note calling ADC_IRQ_Start
 193          *   or ADC_IRQ_StartEx will override any effect this method would 
 194          *   have had. This method should only be called after ADC_IRQ_Start or 
 195          *   ADC_IRQ_StartEx has been called. To set the initial
 196          *   priority for the component use the cydwr file in the tool.
 197          *
 198          * Parameters:
 199          *   priority: Priority of the interrupt. 0 - 7, 0 being the highest.
 200          *
 201          * Return:
 202          *   None
 203          *
 204          *******************************************************************************/
 205          void ADC_IRQ_SetPriority(uint8 priority) 
 206          {
 207   1          *ADC_IRQ_INTC_PRIOR = priority << 5;
 208   1      }
 209          
 210          
 211          /*******************************************************************************
 212          * Function Name: ADC_IRQ_GetPriority
 213          ********************************************************************************
 214          *
 215          * Summary:
 216          *   Gets the Priority of the Interrupt.
 217          *
 218          * Parameters:
 219          *   None
 220          *
 221          * Return:
 222          *   Priority of the interrupt. 0 - 7, 0 being the highest.
 223          *
 224          *******************************************************************************/
 225          uint8 ADC_IRQ_GetPriority(void) 
 226          {
 227   1          uint8 priority;
 228   1      
 229   1      
 230   1          priority = *ADC_IRQ_INTC_PRIOR >> 5;
 231   1      
 232   1          return priority;
 233   1      }
 234          
 235          
 236          /*******************************************************************************
 237          * Function Name: ADC_IRQ_Enable
 238          ********************************************************************************
 239          *
C51 COMPILER V9.51   ADC_IRQ                                                               01/03/2014 20:23:49 PAGE 5   

 240          * Summary:
 241          *   Enables the interrupt.
 242          *
 243          * Parameters:
 244          *   None
 245          *
 246          * Return:
 247          *   None
 248          *
 249          *******************************************************************************/
 250          void ADC_IRQ_Enable(void) 
 251          {
 252   1          /* Enable the general interrupt. */
 253   1          *ADC_IRQ_INTC_SET_EN = ADC_IRQ__INTC_MASK;
 254   1      }
 255          
 256          
 257          /*******************************************************************************
 258          * Function Name: ADC_IRQ_GetState
 259          ********************************************************************************
 260          *
 261          * Summary:
 262          *   Gets the state (enabled, disabled) of the Interrupt.
 263          *
 264          * Parameters:
 265          *   None
 266          *
 267          * Return:
 268          *   1 if enabled, 0 if disabled.
 269          *
 270          *******************************************************************************/
 271          uint8 ADC_IRQ_GetState(void) 
 272          {
 273   1          /* Get the state of the general interrupt. */
 274   1          return ((*ADC_IRQ_INTC_SET_EN & (uint8)ADC_IRQ__INTC_MASK) != 0u) ? 1u:0u;
 275   1      }
 276          
 277          
 278          /*******************************************************************************
 279          * Function Name: ADC_IRQ_Disable
 280          ********************************************************************************
 281          *
 282          * Summary:
 283          *   Disables the Interrupt.
 284          *
 285          * Parameters:
 286          *   None
 287          *
 288          * Return:
 289          *   None
 290          *
 291          *******************************************************************************/
 292          void ADC_IRQ_Disable(void) 
 293          {
 294   1          /* Disable the general interrupt. */
 295   1          *ADC_IRQ_INTC_CLR_EN = ADC_IRQ__INTC_MASK;
 296   1      }
 297          
 298          
 299          /*******************************************************************************
 300          * Function Name: ADC_IRQ_SetPending
 301          ********************************************************************************
C51 COMPILER V9.51   ADC_IRQ                                                               01/03/2014 20:23:49 PAGE 6   

 302          *
 303          * Summary:
 304          *   Causes the Interrupt to enter the pending state, a software method of
 305          *   generating the interrupt.
 306          *
 307          * Parameters:
 308          *   None
 309          *
 310          * Return:
 311          *   None
 312          *
 313          *******************************************************************************/
 314          void ADC_IRQ_SetPending(void) 
 315          {
 316   1          *ADC_IRQ_INTC_SET_PD = ADC_IRQ__INTC_MASK;
 317   1      }
 318          
 319          
 320          /*******************************************************************************
 321          * Function Name: ADC_IRQ_ClearPending
 322          ********************************************************************************
 323          *
 324          * Summary:
 325          *   Clears a pending interrupt.
 326          *
 327          * Parameters:
 328          *   None
 329          *
 330          * Return:
 331          *   None
 332          *
 333          *******************************************************************************/
 334          void ADC_IRQ_ClearPending(void) 
 335          {
 336   1          *ADC_IRQ_INTC_CLR_PD = ADC_IRQ__INTC_MASK;
 337   1      }
 338          
 339          #endif /* End check for removal by optimization */
 340          
 341          
 342          /* [] END OF FILE */
C51 COMPILER V9.51   ADC_IRQ                                                               01/03/2014 20:23:49 PAGE 7   

ASSEMBLY LISTING OF GENERATED OBJECT CODE


             ; FUNCTION ADC_IRQ_Start (BEGIN)
                                           ; SOURCE LINE # 46
                                           ; SOURCE LINE # 47
                                           ; SOURCE LINE # 49
0000 120000      R     LCALL   ADC_IRQ_Disable
                                           ; SOURCE LINE # 52
0003 7E00        R     MOV     R6,#HIGH ADC_IRQ_Interrupt
0005 7F00        R     MOV     R7,#LOW ADC_IRQ_Interrupt
0007 120000      R     LCALL   _ADC_IRQ_SetVector
                                           ; SOURCE LINE # 55
000A 7F07              MOV     R7,#07H
000C 120000      R     LCALL   _ADC_IRQ_SetPriority
                                           ; SOURCE LINE # 58
000F 120000      R     LCALL   ADC_IRQ_Enable
                                           ; SOURCE LINE # 59
0012 22                RET     
             ; FUNCTION ADC_IRQ_Start (END)

             ; FUNCTION _ADC_IRQ_StartEx (BEGIN)
                                           ; SOURCE LINE # 76
0000 900000      R     MOV     DPTR,#address
0003 EE                MOV     A,R6
0004 F0                MOVX    @DPTR,A
0005 A3                INC     DPTR
0006 EF                MOV     A,R7
0007 F0                MOVX    @DPTR,A
                                           ; SOURCE LINE # 77
                                           ; SOURCE LINE # 79
0008 120000      R     LCALL   ADC_IRQ_Disable
                                           ; SOURCE LINE # 82
000B 900000      R     MOV     DPTR,#address
000E E0                MOVX    A,@DPTR
000F FE                MOV     R6,A
0010 A3                INC     DPTR
0011 E0                MOVX    A,@DPTR
0012 FF                MOV     R7,A
0013 120000      R     LCALL   _ADC_IRQ_SetVector
                                           ; SOURCE LINE # 85
0016 7F07              MOV     R7,#07H
0018 120000      R     LCALL   _ADC_IRQ_SetPriority
                                           ; SOURCE LINE # 88
001B 120000      R     LCALL   ADC_IRQ_Enable
                                           ; SOURCE LINE # 89
001E 22                RET     
             ; FUNCTION _ADC_IRQ_StartEx (END)

             ; FUNCTION ADC_IRQ_Stop (BEGIN)
                                           ; SOURCE LINE # 106
                                           ; SOURCE LINE # 107
                                           ; SOURCE LINE # 109
0000 120000      R     LCALL   ADC_IRQ_Disable
                                           ; SOURCE LINE # 110
0003 22                RET     
             ; FUNCTION ADC_IRQ_Stop (END)

             ; FUNCTION ADC_IRQ_Interrupt (BEGIN)
                                           ; SOURCE LINE # 129
                                           ; SOURCE LINE # 142
0000 32                RETI    
C51 COMPILER V9.51   ADC_IRQ                                                               01/03/2014 20:23:49 PAGE 8   

             ; FUNCTION ADC_IRQ_Interrupt (END)

             ; FUNCTION _ADC_IRQ_SetVector (BEGIN)
                                           ; SOURCE LINE # 161
0000 900000      R     MOV     DPTR,#address
0003 EE                MOV     A,R6
0004 F0                MOVX    @DPTR,A
0005 A3                INC     DPTR
0006 EF                MOV     A,R7
0007 F0                MOVX    @DPTR,A
                                           ; SOURCE LINE # 162
                                           ; SOURCE LINE # 163
0008 7B02              MOV     R3,#02H
000A 7A44              MOV     R2,#044H
000C 793A              MOV     R1,#03AH
000E 900000      R     MOV     DPTR,#address
0011 E0                MOVX    A,@DPTR
0012 FE                MOV     R6,A
0013 A3                INC     DPTR
0014 E0                MOVX    A,@DPTR
0015 FF                MOV     R7,A
0016 AD07              MOV     R5,AR7
0018 AC06              MOV     R4,AR6
001A 120000      E     LCALL   _cywrite16_nodpx
                                           ; SOURCE LINE # 164
001D 22                RET     
             ; FUNCTION _ADC_IRQ_SetVector (END)

             ; FUNCTION ADC_IRQ_GetVector (BEGIN)
                                           ; SOURCE LINE # 181
                                           ; SOURCE LINE # 182
                                           ; SOURCE LINE # 183
0000 7B02              MOV     R3,#02H
0002 7A44              MOV     R2,#044H
0004 793A              MOV     R1,#03AH
0006 120000      E     LCALL   _cyread16_nodpx
                                           ; SOURCE LINE # 184
0009         ?C0006:
0009 22                RET     
             ; FUNCTION ADC_IRQ_GetVector (END)

             ; FUNCTION _ADC_IRQ_SetPriority (BEGIN)
                                           ; SOURCE LINE # 205
0000 900000      R     MOV     DPTR,#priority
0003 EF                MOV     A,R7
0004 F0                MOVX    @DPTR,A
                                           ; SOURCE LINE # 206
                                           ; SOURCE LINE # 207
0005 900000      R     MOV     DPTR,#priority
0008 E0                MOVX    A,@DPTR
0009 FF                MOV     R7,A
000A EF                MOV     A,R7
000B C4                SWAP    A
000C 33                RLC     A
000D 54E0              ANL     A,#0E0H
000F FF                MOV     R7,A
0010 90449D            MOV     DPTR,#0449DH
0013 EF                MOV     A,R7
0014 F0                MOVX    @DPTR,A
                                           ; SOURCE LINE # 208
0015 22                RET     
             ; FUNCTION _ADC_IRQ_SetPriority (END)
C51 COMPILER V9.51   ADC_IRQ                                                               01/03/2014 20:23:49 PAGE 9   


             ; FUNCTION ADC_IRQ_GetPriority (BEGIN)
                                           ; SOURCE LINE # 225
                                           ; SOURCE LINE # 226
                                           ; SOURCE LINE # 230
0000 90449D            MOV     DPTR,#0449DH
0003 E0                MOVX    A,@DPTR
0004 FF                MOV     R7,A
0005 EF                MOV     A,R7
0006 C4                SWAP    A
0007 13                RRC     A
0008 5407              ANL     A,#07H
000A FF                MOV     R7,A
000B 900000      R     MOV     DPTR,#priority
000E EF                MOV     A,R7
000F F0                MOVX    @DPTR,A
                                           ; SOURCE LINE # 232
0010 900000      R     MOV     DPTR,#priority
0013 E0                MOVX    A,@DPTR
0014 FF                MOV     R7,A
                                           ; SOURCE LINE # 233
0015         ?C0008:
0015 22                RET     
             ; FUNCTION ADC_IRQ_GetPriority (END)

             ; FUNCTION ADC_IRQ_Enable (BEGIN)
                                           ; SOURCE LINE # 250
                                           ; SOURCE LINE # 251
                                           ; SOURCE LINE # 253
0000 9044C3            MOV     DPTR,#044C3H
0003 7420              MOV     A,#020H
0005 F0                MOVX    @DPTR,A
                                           ; SOURCE LINE # 254
0006 22                RET     
             ; FUNCTION ADC_IRQ_Enable (END)

             ; FUNCTION ADC_IRQ_GetState (BEGIN)
                                           ; SOURCE LINE # 271
                                           ; SOURCE LINE # 272
                                           ; SOURCE LINE # 274
0000 9044C3            MOV     DPTR,#044C3H
0003 E0                MOVX    A,@DPTR
0004 FF                MOV     R7,A
0005 EF                MOV     A,R7
0006 30E504            JNB     ACC.5,?C0010
0009 7F01              MOV     R7,#01H
000B 8002              SJMP    ?C0011
000D         ?C0010:
000D 7F00              MOV     R7,#00H
000F         ?C0011:
                                           ; SOURCE LINE # 275
000F         ?C0012:
000F 22                RET     
             ; FUNCTION ADC_IRQ_GetState (END)

             ; FUNCTION ADC_IRQ_Disable (BEGIN)
                                           ; SOURCE LINE # 292
                                           ; SOURCE LINE # 293
                                           ; SOURCE LINE # 295
0000 9044CB            MOV     DPTR,#044CBH
0003 7420              MOV     A,#020H
0005 F0                MOVX    @DPTR,A
C51 COMPILER V9.51   ADC_IRQ                                                               01/03/2014 20:23:49 PAGE 10  

                                           ; SOURCE LINE # 296
0006 22                RET     
             ; FUNCTION ADC_IRQ_Disable (END)

             ; FUNCTION ADC_IRQ_SetPending (BEGIN)
                                           ; SOURCE LINE # 314
                                           ; SOURCE LINE # 315
                                           ; SOURCE LINE # 316
0000 9044D3            MOV     DPTR,#044D3H
0003 7420              MOV     A,#020H
0005 F0                MOVX    @DPTR,A
                                           ; SOURCE LINE # 317
0006 22                RET     
             ; FUNCTION ADC_IRQ_SetPending (END)

             ; FUNCTION ADC_IRQ_ClearPending (BEGIN)
                                           ; SOURCE LINE # 334
                                           ; SOURCE LINE # 335
                                           ; SOURCE LINE # 336
0000 9044DB            MOV     DPTR,#044DBH
0003 7420              MOV     A,#020H
0005 F0                MOVX    @DPTR,A
                                           ; SOURCE LINE # 337
0006 22                RET     
             ; FUNCTION ADC_IRQ_ClearPending (END)



MODULE INFORMATION:   STATIC OVERLAYABLE
   CODE SIZE        =    183    ----
   CONSTANT SIZE    =   ----    ----
   XDATA SIZE       =   ----       6
   PDATA SIZE       =   ----    ----
   DATA SIZE        =   ----    ----
   IDATA SIZE       =   ----    ----
   BIT SIZE         =   ----    ----
   EDATA SIZE       =   ----    ----
   HDATA SIZE       =   ----    ----
   XDATA CONST SIZE =   ----    ----
   FAR CONST SIZE   =   ----    ----
END OF MODULE INFORMATION.


C51 COMPILATION COMPLETE.  0 WARNING(S),  0 ERROR(S)
